:020000040000FA
:04000000FBEF0DF015
:08000800056ED8CF06F0E0CF31
:1000100007F00001E9CF0DF0EACF08F0E1CF09F0D9
:10002000E2CF0AF0D9CF0BF0DACF0CF0F3CF14F017
:10003000F4CF15F0FACF16F000C00FF001C010F0A9
:1000400002C011F003C012F004C013F0F2AA2CEFAA
:1000500000F0F2B4C5EF01F00FC000F010C001F0E5
:1000600011C002F012C003F013C004F00E8E0DC0D8
:10007000E9FF08C0EAFF09C0E1FF0AC0E2FF0BC0C8
:10008000D9FF0CC0DAFF14C0F3FF15C0F4FF16C08F
:10009000FAFF055007C0E0FF06C0D8FF10000DAE04
:1000A00003D0F2CF0EF0F29EF76AC00FF66E000E8C
:1000B000F7220900F5500DAE02D00EBEF28E1200EE
:1000C00053EF6EF0000000000DAE03D0F2CF0EF043
:1000D000F29EF76AEA0FF66E000EF7220900F5505D
:1000E0000DAE02D00EBEF28E120053EF6EE800008D
:1000F00000000DAE03D0F2CF0EF0F29EF76A140F9F
:10010000F66E010EF7220900F5500DAE02D00EBEBC
:10011000F28E120045786974000000000301716BD3
:100120007151070815E370AF03D093928A8202D011
:1001300093928A9200D000D093948A8400D000D009
:10014000D890703793948A9400D000D0712BE8D760
:1001500093928A8200D000D00001000C93968A9678
:10016000020E0301706F0001D9DF6BC370F3D6DF9D
:100170006DC36EF303016F6B6DC370F30001CEDFCF
:100180006CC370F3CBDF93968A86000C03016B6B14
:100190006D6B040E6C6F0001E1DF550E006E002EDA
:1001A000FED703016B6B6D6B6C6B0001D7DF938C1B
:1001B00081ACFDD7030E03016B6F980E6D6F6C6BF6
:1001C0000001CCDF550E006E002EFED70301666BDA
:1001D00019C065F319C068F3676B036A195067119A
:1001E000696F035019106A6F0B0E6B6F6AC36DF362
:1001F00069C36CF30001B2DF550E006E002EFED70E
:10020000000C030EEA6E650EE96EEF500EE00C0E68
:10021000016E006A002EFED7012EFBD7F70E006E8E
:10022000002EFED700D0EF2EF2D7000CF29CF29EEB
:10023000F2BEFDD7ABDF03016B6B6D6B200E6C6FF5
:1002400000018CDF550E006E002EFED7C00EF2129C
:1002500003016053D8B493D05F532BE0616B6151BD
:10026000070826E3036A6151F2CF65F3F29E0001AD
:1002700016DF030165BFF28E646F93988A88626B04
:100280006251070811E364AF03D093928A8202D0CF
:1002900093928A92939A8A8AD8906437939A8A9A88
:1002A00093988A98622BECD793928A82612BD7D746
:1002B0002AD0616B6151070826E3036A6151F2CFCE
:1002C00065F3F29E000100DF030165BFF28E646FEB
:1002D00093988A88626B6251070811E364AF03D078
:1002E00093928A8202D093928A92939A8A8AD89021
:1002F0006437939A8A9A93988A98622BECD7939250
:100300008A82612BD7D7320E656F00017ADF030135
:10031000636B635101082CE3616B6151070826E3AD
:10032000036A6151F2CF65F3F29E0001E2DE030140
:1003300065BFF28E646F93988A88626B625107087A
:1003400011E364AF03D093928A8202D093928A928F
:10035000939A8A8AD8906437939A8A9A93988A98BB
:10036000622BECD793928A82612BD7D7632BD1D79C
:10037000320E656F000145DF030160076AD76B6BC2
:100380006D6B6C6B0001EADE000CEC0ED76E780E24
:10039000D66E928280B216D01F2A1F3C02D0FE0E6B
:1003A0001F6E1F507D0808E103015F6B010E606F37
:1003B00000013CDF010E1D6E1F50060802E2010E17
:1003C0001E6E01D01F6A928680B610D0212A213C71
:1003D00002D0FE0E216E21507D0802E1010E276E33
:1003E0002150060802E2010E206E03D0216A206A25
:1003F000276A928480B410D0232A233C02D0FE0EB8
:10040000236E23507D0802E1010E286E235006085A
:1004100002E2010E226E03D0236A226A286A9288C1
:1004200080B812D01A2A1A50100801E21A6A1A501B
:10043000060809E1040E19261950D00802E2D00E70
:10044000196E010E1C6E01D01A6A928A80BA12D0FF
:100450001B2A1B50200801E21B6A1B50060809E1F9
:10046000040E195E19500F0802E3100E196E010EEA
:100470001C6E01D01B6A26520BE0252A255013085A
:1004800007E2245202E0246A02D0010E246E256A9B
:10049000F2942CEF00F00301506B5051070811E368
:1004A00094928B824FAF03D094928B8202D094921D
:1004B0008B9294948B94D8904F3794948B84502B38
:1004C000ECD794928B920001000C03014A6B94923A
:1004D0008B824B6B4B51070811E394948B94000073
:1004E00094948B849486000E82B6010E4A134B516D
:1004F000060802E3D8904A374B2BECD74AC301F0E9
:100500000001000C0301486B476B485107080CE3DE
:100510000001DBDF01C049F30301493D01D004D0F4
:10052000472BD8B4482BF1D7493D01D003D0010E59
:10053000016E47D0425140094A6F4F6F0001ABDF57
:1005400046C34BF303014C6B4D6B4E6B46C34FF3ED
:100550000001A1DF45C34BF346C34CF303014D6BD0
:100560004E6B45C34FF3000196DF44C34BF345C3C5
:100570004CF346C34DF303014E6B44C34FF30001EC
:100580008ADF43C34FF387DF950E03014F6F0001EE
:1005900082DF0301486B476B4851070810E30001F5
:1005A00094DF01C049F303014951FE0801E107D07E
:1005B00049BF01D004D0472BD8B4482BEDD749C34D
:1005C00001F00001000C94908B800201F26BF2515B
:1005D000310808E3FF0E03014F6F00015CDF0201E9
:1005E000F22BF5D794908B900301426B466B456BD1
:1005F000446B436B000186DF0201F22D01D00FD066
:10060000F23D01D00CD00301426B466B456B446B4D
:10061000436B000177DF01C0F2F2EED70201F22D49
:100620000DD0010E0301426F466B456B446B436B6B
:10063000000168DF01C0F2F20201F1D7F2C201F05D
:10064000000185EF0EF0186AF2BE188EF29E640E5D
:100650000301656F0001D5DD18BEF28E0201F25371
:100660006EE0F2CFF4F2F29E020EA96EA69CA69E58
:10067000A680A850F4BFF28EF36FEF51F35D16E041
:10068000020EA96EEFC2A8FFA69CA69EA684F2CF7A
:1006900000F0F29E0F01550EA76EAA0EA76EA6825D
:1006A000A6B2FED7A6940050F2120201F2CFF4F2E5
:1006B000F29E010EA96EA69CA69EA680A850F4BF2D
:1006C000F28EF36FEE51F35D16E0010EA96EEEC2ED
:1006D000A8FFA69CA69EA684F2CF00F0F29E0F0172
:1006E000550EA76EAA0EA76EA682A6B2FED7A69436
:1006F0000050F2120201F2CFF4F2F29EA96AA69C17
:10070000A69EA680A850F4BFF28EF36F1950F35D39
:1007100015E0A96A19C0A8FFA69CA69EA684F2CFE0
:1007200000F0F29E0F01550EA76EAA0EA76EA682CC
:10073000A6B2FED7A6940050F212020129D0010EF3
:10074000A96EA86AA69CA69EA684F2CF00F0F29E8F
:100750000F01550EA76EAA0EA76EA682A6B2FED7EF
:10076000A6940050F212020EA96E010EA86EA69C6D
:10077000A69EA684F2CF00F0F29E550EA76EAA0E9A
:10078000A76EA682A6B2FED7A6940050F21202016E
:10079000186AF2BE188EF29E640E0301656F0001A6
:1007A00030DD18BEF28E939E8A9E186AF2BE188EB5
:1007B000F29E640E0301656F000123DD18BEF28E08
:1007C000949A8B9A94988B980300000C0301416BC8
:1007D000415163083BE394908B90110E426F3CC3F0
:1007E00046F33BC345F33AC344F339C343F3000133
:1007F00089DE01C03FF303013F5319E13E6B3D6BBE
:100800003E51130813E303E13D5187080FE3000154
:100810005CDE01C040F303014051FE0803E1000E1D
:10082000016E16D03D2BD8B43E2BEAD70DD03F51E8
:10083000FE0803E1000E016E0BD094908B800A0E2F
:10084000006E002EFED70000412BC2D7010E016EB4
:100850000001000C3ADE39DE0301226B216B2251CC
:1008600007080CE3000131DE013C03D0030106D090
:1008700000010301212BD8B4222BF1D70001000C79
:1008800003011D6B1551FE0B1E6F16C31FF317C31B
:1008900020F317C33CF316C33BF33A6F1DC339F380
:1008A000000194DF015201E037D0030114C31AF3B1
:1008B0001551010B1B6F196B186B195101082AE3B5
:1008C0001A51185D20E11B51195D1DE11C6B1C5173
:1008D0001F0818E3036A1C512C0F016E000E03223F
:1008E00001C01DF303C01EF30001EFDD1EC3EAFFCC
:1008F0001DC3E9FF01C0EFFF0301182BD8B4192B6A
:100900001C2BE5D703D00001E0DD0301182BD8B480
:10091000192BD3D700019EDF000C03013C6B3D6B0C
:10092000010E3E6FDA6AD96A030E416F340E406FD2
:10093000030EEA6E380EE96E41C3E2FF40C3E1FFE9
:100940003EC33FF3D890E550EE02F3503C23F45001
:100950003D233F2FF7D73CC3DEFF3DC33CF33D6B48
:10096000D8B03D2B402BD8B4412B3E2B3E5105082F
:10097000DFE10001000C006A016A026A036A0301F8
:10098000146B156B166B176B13511211111110119B
:100990002CE0200E186FD8900C370D370E370F371C
:1009A00014371537163717371351175D08E11251F1
:1009B000165D05E11151155D02E11051145D0FE363
:1009C0001051145F1151D8A0113D155F1251D8A0DC
:1009D000123D165F1351D8A0133D175FD880003623
:1009E000013602360336182FD6D7030EEA6E140EE0
:1009F000E96E0001F3EF06F00301176B166B010EB1
:100A0000156FBE0E146F00013BDF0301036B026B19
:100A1000016B066B056B06C303F005C302F0006AA9
:100A2000005034240201F66F355003010121020108
:100A3000F76F0250030102210201F86F0350030116
:100A400003210201F96FD8900301006B0201F63512
:100A50000301016F0201F7350301026F0201F8354E
:100A60000301036F176F02C316F301C315F300C32D
:100A700014F3000105DF0301036B026B016B066BCE
:100A8000056B06C303F005C302F0006A005037246B
:100A90000201FA6F3850030101210201FB6F02507D
:100AA000030102210201FC6F035003010321020133
:100AB000FD6FFA5307E1FB51020804E1FC5302E128
:100AC000FD5303E0010E016EA5D139C0ACF03AC070
:100AD00000F0016A026A036A3A50F6250301006FCA
:100AE00001500201F7210301016F02500201F821B8
:100AF0000301026F03500201F9210301036F066B2A
:100B0000056B06C303F005C302F0006A0050002520
:100B10000001B16F3B50030101210001B26F02508F
:100B2000030102210001B36F0350030103210001FF
:100B3000B46F0301036B026B016B066B056B06C39D
:100B400003F005C302F0006A00503D240001AD6FC0
:100B50003E50030101210001AE6F0250030102214A
:100B60000001AF6F0350030103210001B06F0301C7
:100B7000036B026B016B066B056B06C303F005C3C9
:100B800002F0006A005042240201FA6F4350030150
:100B900001210201FB6F0250030102210201FC6FDF
:100BA0000350030103210201FD6FFA5309E1FB53D6
:100BB00007E1FC5305E1FD5303E1010E016E2AD16B
:100BC0000301036B026B016B3CC000F303C337F3FB
:100BD00002C336F301C335F33CC034F3FDC23BF32B
:100BE000FCC23AF3FBC239F3FAC238F3000195DED6
:100BF0000050B125B56F0150B221B66F0250B3213C
:100C0000B76F0350B421B86FB0310201FD6F00011E
:100C1000AF310201FC6F0001AE310201FB6F000138
:100C2000AD310201FA6FFD33FC33FB33FA33FD3390
:100C3000FC33FB33FA33FD33FC33FB33FA330F0E53
:100C4000FD170001AD510F0B006E016A026A036AC5
:100C5000005206E1015204E1025202E1035209E0AE
:100C6000010E0201FA27D8B0FB2BD8B4FC2BD8B464
:100C7000FD2B0201FA510001B525B96F0201FB51AC
:100C80000001B621BA6F0201FC510001B721BB6F10
:100C90000201FD510001B821BC6F0301036B026B1F
:100CA000016B066B056B06C303F005C302F0006A17
:100CB00000503F240201F26F405003010121020164
:100CC000F36F0250030102210201F46F035003018C
:100CD00003210201F56FF25366E1F35364E1F4532B
:100CE00062E1F55360E1D8900301006B0201F63533
:100CF0000301016F0201F7350301026F0201F835AC
:100D00000301036F200E0025046F000E0121056F03
:100D1000000E0221066F000E0321076F176F06C336
:100D200016F305C315F304C314F30001A9DD030191
:100D3000036B026B016B066B056B2DC001F0006A43
:100D400000502C24096F2D5001210A6F05510221FA
:100D50000B6F065103210C6F0E6B2EC002F0006A60
:100D6000016A00500925126F01500A21136F2E509D
:100D70000B21146F0E510C21156F006A016A026A73
:100D8000005012250201F26F0150030113210201EC
:100D9000F36F0250030114210201F46F2F5003017D
:100DA00015210201F56F0001B1510201F25F00014E
:100DB000B2510201F35B0001B3510201F45B000187
:100DC000B4510201F55BF5C20FF3F4C20EF3F3C2A6
:100DD0000DF3F2C20CF30301136B126B116BACC079
:100DE00010F30001C8D503C0F5F202C0F4F201C04F
:100DF000F3F200C0F2F20201F55305E1F45303E10E
:100E0000F3510F0804E2000E016E04D003D0010E6E
:100E1000016E00D000019BEF0EF003011E6BD89015
:100E2000186B0001B5350301196F0001B6350301D8
:100E30001A6F0001B73503011B6F176B166B156B2B
:100E4000146B17510001B05DD8A004D116E1030165
:100E500016510001AF5DD8A0FDD00FE1030115517F
:100E60000001AE5DD8A0F6D008E1AD510301145DDC
:100E7000D8A002D00001EED000011BC33CF31AC37E
:100E80003BF319C33AF318C339F3A0DC015204E071
:100E900003011EC301F0E1D003011C6B1C510F08BC
:100EA000D8A0C7D01D6B1D511F0816E3036A1D5142
:100EB0002C0F016E000E032201C01FF303C020F3AC
:100EC000000165EC02F020C3EAFF1FC3E9FF01C087
:100ED000EFFF03011D2BE7D72C5201E1AAD04652A8
:100EE00003E14752D8B49BD02C50E508D8B497D032
:100EF00037501008D8A493D01E2B132F90D0226BFC
:100F0000216B206B46C01FF3266B256B246B47C0FB
:100F100023F325C303F024C302F047C001F0006AA5
:100F200000504624286F47502021296F2451212149
:100F30002A6F255122212B6F020E285D2C6F000E87
:100F400029592D6F000E2A592E6F000E2B592F6F25
:100F5000ACC000F0016A026A036A03C033F302C046
:100F600032F301C031F3ACC030F3376F2EC336F328
:100F70002DC335F32CC334F303C03BF302C03AF363
:100F800001C039F3ACC038F30001C7DC03C030F353
:100F900002C02FF301C02EF300C02DF3B95103019D
:100FA0000024316F0001BA5103010120326F0001AA
:100FB000BB5103010220336F0001BC510301032028
:100FC000346FD890356B3135366F3235376F3335F6
:100FD000386F3C6F37C33BF336C33AF335C339F34D
:100FE0000001E6EC03F003011D6B1D511F0816E321
:100FF000036A1D512C0F016E000E032201C01FF366
:1010000003C020F3000165EC02F020C3EAFF1FC318
:10101000E9FF01C0EFFF03011D2BE7D70AD0010E46
:101020001427D8B0152BD8B4162BD8B4172B1C2BDB
:1010300035D700010FDC2C5201E10CD00301135312
:1010400003E1000107D00301020E1927000E1A2345
:101050001B23F7D603011EC301F00001000C03019E
:101060001E6BD890186B0001B5350301196F000194
:10107000B63503011A6F0001B73503011B6F176BFB
:10108000166B156B146B17510001B05DD8A07CD0A6
:1010900016E1030116510001AF5DD8A075D00FE134
:1010A000030115510001AE5DD8A06ED008E1AD512D
:1010B0000301145DD8A002D0000166D000011BC35B
:1010C0003CF31AC33BF319C33AF318C339F3E6EC04
:1010D00003F0015204E003011EC301F058D00301E4
:1010E0001C6B1C510F083EE31D6B1D511F0816E3BE
:1010F000036A1D512C0F016E000E032201C01FF365
:1011000003C020F3000165EC02F020C3EAFF1FC317
:10111000E9FF01C0EFFF03011D2BE7D72C5201E1CE
:1011200021D0465202E1475213E02C50E50810E06E
:101130003750180B0DE134504D080AE13550500876
:1011400007E13650330804E11E2B132F01D00AD0DB
:10115000010E1427D8B0152BD8B4162BD8B4172BE2
:101160001C2BBFD700012AEC04F02C5201E10CD05B
:101170000301135303E1000107D00301020E1927F5
:10118000000E1A231B237FD703011EC301F00001A9
:10119000000C03011E6B226B216B206B46C01FF3FA
:1011A000266B256B246B47C023F325C303F024C3B0
:1011B00002F047C001F0006A00504624286F4750F3
:1011C0002021296F245121212A6F255122212B6FA3
:1011D000020E285D2C6F000E29592D6F000E2A5922
:1011E0002E6F000E2B592F6FACC000F0016A026AFF
:1011F000036A03C033F302C032F301C031F3ACC061
:1012000030F3376F2EC336F32DC335F32CC334F3CD
:1012100003C03BF302C03AF301C039F3ACC038F36A
:1012200000018DEC04F0B95103010024316F00017D
:10123000BA5103010120326F0001BB5103010220AA
:10124000336F0001BC5103010320D890186B313576
:10125000196F32351A6F33351B6F176B166B156BA1
:10126000146B17510001B05DD8A07CD016E10301CA
:1012700016510001AF5DD8A075D00FE103011551E3
:101280000001AE5DD8A06ED008E1AD510301145D40
:10129000D8A002D0000166D000011BC33CF31AC3E2
:1012A0003BF319C33AF318C339F3E6EC03F00152E8
:1012B00004E003011EC301F058D003011C6B1C5154
:1012C0000F083EE31D6B1D511F0816E3036A1D51F5
:1012D0002C0F016E000E032201C01FF303C020F388
:1012E000000165EC02F020C3EAFF1FC3E9FF01C063
:1012F000EFFF03011D2BE7D72C5201E121D046520D
:1013000002E1475213E02C50E50810E03750180B6B
:101310000DE134504D080AE13550500807E13650D0
:10132000330804E11E2B132F01D00AD0010E14271D
:10133000D8B0152BD8B4162BD8B4172B1C2BBFD76D
:1013400000012AEC04F02C5201E10CD003011353EC
:1013500003E1000107D00301020E1927000E1A2332
:101360001B237FD703011EC301F00001000CCDC277
:10137000F3F20201F46BF26BF2511F080AE3036A05
:10138000F251CE0FE96E020E0320EA6EEF6AF22BE5
:10139000F3D7FF0E0301136F000161DE01C0CEF22F
:1013A000010E0201F26FF2511F0825E3F35301E130
:1013B00022D0F42BF4C213F300012FDD036A0201E3
:1013C000F251CE0F016E020E032201C0F5F203C0EE
:1013D000F6F2FF0E0301136F0001DBDEF6C2EAFF37
:1013E000F5C2E9FF01C0EFFF0201F351F45D01E135
:1013F00002D0F22BD8D70001BAEF0EF00201F46B45
:10140000F36BF26BF2511F080EE3036AF251CE0F39
:10141000E96E020E0320EA6EEF50036AF3270350D1
:10142000F423F22BEFD7F35306E1F45304E1000E5B
:10143000016E04D003D0010E016E00D00001BCEF9C
:101440000EF00201EE51CD5D03E2000E016E12D0EE
:10145000036AEE51CE0FE96E020E0320EA6EEF50E2
:10146000EF5D05E004E3000E016E04D003D0010E31
:10147000016E00D00001FFEF0EF00201EE51CD5DD4
:1014800001E2EE6BF26B010ECD25F26FF25315E027
:10149000036AEE51CE0FE96E020E0320EA6EEF52A0
:1014A00006E1EE2BEE51CD5D01E2EE6B04D0010EB4
:1014B000EF6F016E04D0F22BE6D7000E016E000133
:1014C000000C000E016EC250C70B0110C26EC28428
:1014D000C2B4FED7C3CF29F0C4CF2AF02A5229E1E3
:1014E00029509D0826E32A5217E129509A0814E34F
:1014F000186AF2BE188EF29E03015F6B050E606FD4
:10150000000116EC01F018BEF28E010E0201F26F1E
:10151000000123EC03F00DD0186AF2BE188EF29E83
:1015200003015F6B020E606F000116EC01F018BE44
:10153000F28E000C0301125306E111C313F30001F4
:101540008EDD08D0030112C313F3000166DC11C362
:1015500013F31FDE72EF0BF0030117C31DF31851D5
:10156000010B1E6F176B18910001C9510301175D24
:101570000FE10001CA510301185D0AE10001CB51DE
:101580000301195D05E10001CC5103011A5D3CE046
:101590001AC33CF319C33BF318C33AF317C339F327
:1015A0000001E6EC03F0015204E0000E016E026E51
:1015B0004BD00301206BCD0E1F6F2051020818E3A2
:1015C00003E11F51CC0814E320C303F01F511F2B6C
:1015D000D8B4202B216F03C022F3000165EC02F088
:1015E00022C3EAFF21C3E9FF01C0EFFF0301E5D7F2
:1015F00000012AEC04F01AC3CCF019C3CBF018C3D5
:10160000CAF017C3C9F003011EC303F01D511D2BFF
:10161000D8B41E2B216FCD0E2125E96E000E0320BC
:10162000EA6EEF501C6B1B6FCD0E1D25E96E000E90
:101630001E21EA6EEF50216F000E1B1321511C1367
:101640001BC301F01CC302F0000157EF0BF0D89050
:101650000301176B0001B1350301186F0001B235AA
:101660000301196F0001B33503011A6F1E6B1D6B67
:10167000D8901135006E1235016E1D35026E1E3583
:10168000036E00501725136F01501821146F02507C
:101690001921156F03501A21166F16C31AF315C3BB
:1016A00019F314C318F313C317F3000155D702C07D
:1016B00012F301C011F303011251FE0808E2FF0A00
:1016C00003E11151F70803E2FF0E126F116F11C30E
:1016D00001F012C302F00001000CF2C211F3EEC2DD
:1016E00012F328D70301066B056B046B096B086BBB
:1016F00049C001F0006A005048240C6F4950042191
:101700000D6F085105210E6F095106210F6F116BE6
:101710004AC002F0006A016A00500C25156F0150A2
:101720000D21166F4A500E21176F11510F21186F9E
:10173000006A016A026A005015250001C16F01505C
:10174000030116210001C26F02500301172100019D
:10175000C36F4B50030118210001C46F0301046BD8
:10176000000E46240001BD6F475003010421000113
:10177000BE6FD890C86BC431C76FC331C66FC2315A
:10178000C56FC1C0FBF20001C251010B0201FC6F29
:101790000001BD3D03D0BE3D01D005D0BE5306E1E2
:1017A000BD51010803E3090E016EFDD1BEC012F365
:1017B000BDC011F34CDF02C0C0F001C0BFF0020198
:1017C000FE6BACC0FDF20301066B056BBEC004F3FB
:1017D000BDC003F3020E035D076F000E0459086FCE
:1017E000000E0559096F000E06590A6FACC000F0D3
:1017F000016A026A036A03C00EF302C00DF301C05E
:101800000CF3ACC00BF3376F09C336F308C335F3E1
:1018100007C334F303C03BF302C03AF301C039F30A
:10182000ACC038F300018DEC04F0B9510301002481
:101830000C6F0001BA51030101200D6F0001BB5173
:10184000030102200E6F0001BC5103010320D89058
:101850000201F76B03010C350201F86F03010D352E
:101860000201F96F03010E350201FA6F186AF2BE28
:10187000188EF29E0001C6EC00F018BEF28EC55321
:1018800007E1C65305E1C75303E1C853D8B445D1B6
:10189000FAC23CF3F9C23BF3F8C23AF3F7C239F3A8
:1018A000E6EC03F0015203E0090E016E7CD1020167
:1018B000F46BF36BF451010827E3938C81ACFDD7F3
:1018C000000165EC02F001C0FFF293988A880301E1
:1018D000006B0051070813E30201FFAF03D093929E
:1018E0008A8202D093928A92939A8A8AD890FF37FA
:1018F000939A8A9A93988A980301002BEAD7020157
:10190000F32BD8B4F42BD6D71E5236E0938C81AC8F
:10191000FDD7186AF2BE188EF29E010E03015F6FAA
:10192000606F000116EC01F018BEF28E928280A268
:10193000FDD71D5204E0010E016E35D11CD01E6A88
:10194000010E266E1E5208E1245203E0949A8B8AFF
:1019500002D0949A8B9AF6D7949A8B8A928280B20C
:1019600002D01E6AFBD7266A949A8B8A1D5203E026
:10197000010E016E18D10201F29CF29EF2BEFDD75B
:101980001C521FE00301046B19C003F319C006F3D6
:10199000056B036A19500511076F03501910086F82
:1019A000186AF2BE188EF29E0B0E6B6F08C36DF3B1
:1019B00007C36CF30001AEEC00F018BEF28E1C6A97
:1019C00002011D5205E0010E016E0001ECD0020182
:1019D000205208E0938C81ACFDD7020E016E00010D
:1019E000E2D00201225208E0938C81ACFDD7030EB5
:1019F000016E0001D8D00201C00EF212FF0E0001EC
:101A0000C527D8A0C627D8A0C727D8A0C8270201B5
:101A1000FD51D8B4FE07FD2F02D0FE5306E0020EA2
:101A2000F827000EF923FA2376D00001BF530CE10A
:101A3000C0530AE1BEC012F3BDC011F308DE02C0FC
:101A4000BEF001C0BDF006D0C0C0BEF0BFC0BDF04A
:101A5000C06BBF6BBD3D03D0BE3D01D005D0BE53B2
:101A600004E1BD51010801E358D00301066B056B89
:101A7000BEC004F3BDC003F3020E035D076F000E8A
:101A80000459086F000E0559096F000E06590A6FB8
:101A9000ACC000F0016A026A036A03C00EF302C020
:101AA0000DF301C00CF3ACC00BF3376F09C336F371
:101AB00008C335F307C334F303C03BF302C03AF362
:101AC00001C039F3ACC038F300018DEC04F0B9511A
:101AD000030100240C6F0001BA51030101200D6FB6
:101AE0000001BB51030102200E6F0001BC51030134
:101AF0000320D8900201F76B03010C350201F86F47
:101B000003010D350201F96F03010E350201FA6F71
:101B1000FE6BACC0FDF20001B2D60201FB5302E144
:101B2000FC533FE0FAC23CF3F9C23BF3F8C23AF38C
:101B3000F7C239F30001E6EC03F0015203E0090EAD
:101B4000016E31D00201F46BF36BF451FC5D29E3BB
:101B500003E1FB51F35D25E2938C81ACFDD70001DD
:101B600065EC02F001C001F393988A880301026BCF
:101B70000251070811E301AF03D093928A8202D089
:101B800093928A92939A8A8AD8900137939A8A9AE2
:101B900093988A98022BECD70201F32BD8B4F42B3C
:101BA000D4D7000E016E000172EF0FF00201EE3D7E
:101BB00002D0CDC2EEF2F26B010ECD25F26FF253E0
:101BC00015E0036AEE51CE0FE96E020E0320EA6EB5
:101BD000EF5206E1EE07EE3D02D0CDC2EEF204D0A8
:101BE000010EEF6F016E04D0F22BE6D7000E016EEE
:101BF0000001E0EF0FF0F86AD09E0D8EEA6AE96A04
:101C0000C180C182C184C196926A896A936A8A6AD4
:101C1000946A170E8B6EC190C182C184C186C18C3B
:101C2000C29CC28EC18EC2801F0E926E400E936EF9
:101C3000080E946E939E8A9E2B6A94988B88949A31
:101C40008B8A939E8A8E928280A2FDD7928680B6DE
:101C500002D0010E2B6E928680A6FDD71A6A1B6AEF
:101C60001C6A1D6A1E6A1F6A206A216A226A236A28
:101C7000246A256A266A276A286A830ED56EEC0EC6
:101C8000D76E780ED66EF28AC00EF212F2CFF2F252
:101C9000F29EA96AA69CA69EA680A8500201F2BF49
:101CA000F28E196E193C02D0300E196E1950800850
:101CB00002E2600E196EF29CF29EF2BEFDD7186A27
:101CC000F2BE188EF29E0001C6EC00F018BEF28E35
:101CD000C00EF212186AF2BE188EF29EFA0E0301BE
:101CE000656F000101EC01F018BEF28E186AF2BEB9
:101CF000188EF29E010E03015F6F606F000116ECFB
:101D000001F018BEF28EE3EF02F0013C12D0186A27
:101D1000F2BE188EF29E03015F6B080E606F000129
:101D200016EC01F018BEF28E0201F26B000123ECFA
:101D300003F0FCEF04F0015213E0186AF2BE188EB3
:101D4000F29E010E03015F6F080E606F000116EC3A
:101D500001F018BEF28E0201F26B000123EC03F0D9
:101D6000FF0E0301136F00010DEC07F001C0CDF26F
:101D7000B7EF09F0FEEF09F0015213E1186AF2BE65
:101D8000188EF29E010E03015F6F040E606F00015A
:101D900016EC01F018BEF28E0201F26B000123EC8A
:101DA00003F0F2CFF2F2F29E010EA96EA69CA69E5F
:101DB000A680A8500201F2BFF28EEE6FF2CFF2F2CF
:101DC000F29E020EA96EA69CA69EA680A850F2BF07
:101DD000F28EEF6F2B5210E0EE6B010EEF6F186A70
:101DE000F2BE188EF29E010E03015F6F606F00015C
:101DF00016EC01F018BEF28E000121EF0AF001523C
:101E00000CE10201EE6B00013DEC0AF0015205E12C
:101E10000201F26B000123EC03F0020E0201F26FEB
:101E2000186AF2BE188EF29EFA0E0301656F000169
:101E300001EC01F018BEF28E0201F22FF1D792826E
:101E400080B202D01E6AFBD71D5206E0010EF26F6F
:101E5000000123EC03F00201020EF26F186AF2BED9
:101E6000188EF29EFA0E0301656F000101EC01F07D
:101E700018BEF28E0201F22FF1D7928280B202D008
:101E80001E6AFBD71D5205E0010EF26F000123EC24
:101E900003F0000161EC0AF01D5206E0010E0201A0
:101EA000F26F000123EC03F0036A0201EE51CE0F42
:101EB000E96E020E0320EA6EEF50EF5D03E002E3ED
:101EC000010EEF6FEF5309E1036AEE51CE0FE96E99
:101ED000020E0320EA6EEFCFEFF2EFC2F2F2000142
:101EE0006DEF0BF001C0F0F20201F02D06D0010EF3
:101EF000F26F000123EC03F00201F051020834E11B
:101F0000186AF2BE188EF29E010E03015F6F606FB9
:101F1000000116EC01F018BEF28E0201EF2B206AD0
:101F2000928680B621D027521DE0186AF2BE188E24
:101F3000F29E010E03015F6F020E606F000116EC4E
:101F400001F018BEF28E276A206A0201EE2B000112
:101F50003DEC0AF0015205E10201F26B000123ECB5
:101F600003F00201206ADCD7F051030833E1186A5C
:101F7000F2BE188EF29E010E03015F6F606F0001CA
:101F800016EC01F018BEF28E0201EF07226A92846D
:101F900080B420D028521CE0186AF2BE188EF29E3F
:101FA000010E03015F6F020E606F000116EC01F07D
:101FB00018BEF28E286A226A0201EE070001F6D5E9
:101FC000015205E10201F26B000123EC03F0020172
:101FD000226ADDD7F051090826E1F16BF1510308BF
:101FE0001DE3186AF2BE188EF29E03015F6B010EAC
:101FF000606F000116EC01F018BEF28E186AF2BE96
:10200000188EF29E010E03015F6F606F000116ECE7
:1020100001F018BEF28E0201F12BE0D7F26B000145
:1020200023EC03F00201F05301E1EF2B000161EC1E
:062030000AF032D70300A4
:020000040030CA
:0E00000000060E0E000080000FC00FE00F4043
:00000001FF
